:020000040000FA
:10000000000000308A00412817280F398207303459
:10001000313432343334343435343634373438349C
:100020003934413442344334443445344634F000A6
:10003000030EF1000A08F2008A010408F30083129B
:1000400003130C1C2728AB0A0319AC0A0C100B1D58
:1000500036280B11E008031D3028E1080319362863
:10006000E003600A0319E1030319E0088312031394
:100070007308840072088A00710E8300F00E700EFF
:10008000090007308A0018278A0187157E16462541
:100090000815EC210A230910861A4C280914861E1B
:1000A0004F28A901AA0189100810CA247E1124250D
:1000B00003187E157E194829132500302E02031DD2
:1000C000632880302D02000003187628FE1D6B285F
:1000D0002330FE116D282030FE150530F500B030BC
:1000E000E0220530F500BF30E0225628A908031DA4
:1000F00084280530F500D130E022CD21D62205300C
:10010000F500F530E022CA241C248F018E01AB01DA
:10011000AC017E128B170910861A8C280230E10080
:10012000E830E000F0247E11242503187E157E19A6
:100130004829E108031D9228E008031D92280914AC
:10014000861EA0287E168B13D624DF08031D3529B2
:10015000102416240B30BA00EB30B900C230B800BE
:100160000030B7002C08BF002B08BE000F08BD00F0
:100170000E08BC003C08B7023D08031C3D0FB80246
:100180003E08031C3E0FB9023F08031C3F0FBA0292
:10019000BA1F0129B709B809B70A0319B80A00300C
:1001A0003802031DD528643037020000031CDA280A
:1001B00087153529871100303802031DE1281430D6
:1001C000370200000318BB2100303802031DEA2863
:1001D0000F30370200000318BB2100303802031D26
:1001E000F3280A30370200000318BB210030380220
:1001F000031DFC280530370200000318BB21BB217A
:10020000352900303802031D072964303702000009
:10021000031C0C29871535298711B70803193529BF
:1002200000303802031D162914303702000003186D
:10023000C22100303802031D1F290F303702000091
:100240000318C22100303802031D28290A30370262
:1002500000000318C22100303802031D3129053087
:10026000370200000318C221C22100303802031DEA
:100270003B29053037020000031C41290810891072
:100280004329081489141623A90A0319AA0A552810
:10029000D6220630F5000730E0222B2501305E0221
:1002A000031D5B290730F5000830E0220630F50019
:1002B0001930E022CE2102305E02031D9C29063057
:1002C000F5002B30E022DF0A04305F020319DF0162
:1002D000DF08031D7A294625162387110630F5000D
:1002E0007330E022CE210630F5008530E022CA21AD
:1002F000CA214128871501305F02031D8529063078
:10030000F5003D30E0220130A80002305F02031DFD
:100310008F290630F5004F30E0228030A8000330EE
:100320005F02031D99290630F5006130E022FF309D
:10033000A800CD217E114B2803305E02031DA829A1
:100340000630F500A930E022CA245125CD214128EC
:1003500004305E02031DB5290730F5000830E022A5
:100360000630F5009730E022CE217E11DE01D62244
:10037000A901AA014B28A80AA808031DC129FF301A
:10038000A8000800A803A808031DC8290130A80078
:100390000800CA21CE21CE21CE21CE21D121D121CA
:1003A000D121FA30E029C830E0296430E029323028
:1003B000E0290A30E0290530E0290230E029013047
:1003C000A7000430A6003D30A500A50BE529A60B2B
:1003D000E529A70BE129080087120F30E021203022
:1003E000A3228030A3220530E0212030A3228030D8
:1003F000A3220130E021063099220C3099221430DA
:1004000099223522D6220530F5005630E0220530FB
:10041000F5006830E022CD210530F5007A30E02289
:100420000530F5008C30E022CE21D6220800A00055
:10043000AF222008881507128712F039A322200E58
:10044000F039A32AA0000310A00DA00DA00DAF222B
:100450002008403899220830A20042221722F40ACC
:100460000319F50AA20B2D2A08000230F5005930B5
:10047000F4000830A300A40124082222A40AA30B3C
:100480003C2A08008312031774088D0075088F003A
:10049000831603178C178B138B1B4B2A0C1400002D
:1004A00000007E1E8B17831203170C0883120313A0
:1004B00008000034003400341034103400340034A8
:1004C0000034003400340034143414340034003464
:1004D0000034003400340034153415340034003452
:1004E000003400340134013415341534013401343E
:1004F00000340034103410341034103410341034FC
:1005000000340034143414341434143414341434D3
:1005100000340034153415341534153415341534BD
:100520000034FF34FF34FF34FF34FF34FF34FF3432
:10053000FF34A000AF222008881107128712F0397B
:10054000A322200EF039081801388818023808193B
:100550000438881908388800871687120800881719
:1005600083160313881783120313881107167E104E
:100570008716D022881F7E148712D0228716D02299
:100580008712D0227E1CB72A831603138813831286
:100590000313071208000000000000000000000024
:1005A0000000000000000000000008000130992A4F
:1005B0000230992A8030992AC030992A8038992AA5
:1005C000831203178D0075088F00ED22DE22ED22C5
:1005D000FF39031908001722E72A831603178C171F
:1005E0008B138B1BF02A0C14000000007E1E8B174F
:1005F000831203170C088D0A03198F0A8312031341
:1006000008002030172AA100210E052017222108FA
:100610000520172A8312031391010C3097008316CB
:100620000313FF309200071183120313280895006B
:100630000800373084000A30A2002F082202AF00E1
:1006400030082202B0003108A202FE10B0030319E4
:10065000FE14B00AB008031D2F2B2C3017220008FF
:10066000840AA300AF08031D412BFE183E2B303037
:100670002302031D3E2B2030A3003F2BFE14230832
:100680001722AF080319452BAF03B003A20B262B8B
:1006900008001E242830A2003C30C3003230C400C1
:1006A000C1010310BA0CB90CB80CB70C031C712BA8
:1006B0000530A300430884000008C10044088400FA
:1006C0004208C2018007031C672B0130C2004108A9
:1006D0008007031C6D2B0130C200C30AC40AA30BA0
:1006E0005A2B0310BC0DBD0DBE0DBF0DC00DA20BCE
:1006F0004C2B0800A2011E24BC08031D8C2BBD0836
:10070000031D8C2BBE08031D8C2BBF08031D8C2BD7
:10071000C008031D8C2B0800A20A0310C01BB42BB9
:10072000BC0DBD0DBE0DBF0DC00D40083B02031D2D
:10073000AA2B3F083A02031DA92B3E083902031DCC
:10074000A82B3D083802031DA72B3C0837020000E8
:1007500000000000000003188C2B1E240310C00CA6
:10076000BF0CBE0CBD0CBC0C40083B02031DC92BCA
:100770003F083A02031DC82B3E083902031DC72B50
:100780003D083802031DC62B3C083702000000005C
:1007900000000000031CDE2B3C08B7023D08031CD0
:1007A0003D0FB8023E08031C3E0FB9023F08031C70
:1007B0003F0FBA024008031C400FBB02B20DB30D3D
:1007C000B40DB50DB60DA20BAE2B08001E242830BB
:1007D000A2000530A3003230840000080F39C100A8
:1007E00005304102031CF62B033080070008F03966
:1007F000C10050304102031CFF2B30308007840AB7
:10080000A30BED2B0310B70DB80DB90DBA0DBB0D31
:10081000B20DB30DB40DB50DB60DA20BE92B08004A
:10082000B701B801B901BA01BB010800BC01BD01A3
:10083000BE01BF01C001080010241624B201B3019B
:10084000B401B501B60108003308BD003208BC0090
:100850003408BE003508BF003608C0000800330861
:10086000B8003208B7003408B9003508BA003608B5
:10087000BB000800102416243730C3003630C400F3
:100880000530A20044088400000E4E244408840071
:1008900000084E24C403A20B422C08000F39303844
:1008A000C1004308840041088000C30A08001E24D8
:1008B0002830A3000310BB0CBA0CB90CB80CB70C51
:1008C000B60CB50CB40CB30CB20C37308400053048
:1008D000A200801F6D2C30308002801D712C0330EF
:1008E0008002840AA20B692CA30B5A2C08001E2438
:1008F0003730C3003230C4000530A2004308840002
:1009000000080F39A300840A000EF039A30444083C
:10091000840023088000C30AC30AC40AA20B7E2CE9
:100920002F2C831603178C18932C76088312031729
:100930008D0077088C00831603178C130C158B130E
:1009400055308D00AA308D008C147E1E8B170C1133
:100950008312031308008312031776088D00831691
:1009600003178C130C14831203170C088312031340
:1009700008008400AB248000840AF60AA20BBA2C7B
:10098000080084000008F7009124840AF60AA20BEC
:10099000C22C08000530F500E730E0221C242808AE
:1009A000B7000330AF00B001B1010B2D0030DE22E3
:1009B0001C242C08BA002B08B9000F08B8000E0838
:1009C000B7000530BC0049232F240A30AF000230A5
:1009D000B000B1010B25483017227A301722012BC5
:1009E0000E30DE221C246108B8006008B7002530F4
:1009F000BC007A233208DB005C085B0203190A2D75
:100A00005B08DC001E245B08B7000230AF00B001B9
:100A1000B1010B250800E6233A24192B0630F50016
:100A2000BB30E02208008530162D81309F00DF2189
:100A30009F149F18192D831603131E088312031386
:100A4000AD001E08AE00080006080F390F3A031467
:100A50000319031008002425031C2B2DDE010608B2
:100A60000F39A400D92106080F392402031D2E2DA9
:100A7000DE0A241C422DDE0AA41C422DDE0A241D9F
:100A8000422DDE0A24250318422D0800F601AB246E
:100A9000A800FF302802031D502D8030A800512DE2
:100AA0000800F6012808F7009124080000344634B5
:100AB000723465347134753465346E347A346E341E
:100AC0006F3472346D3461346C342034203400342B
:100AD0004034313430344D3448347A342034203486
:100AE00028346334293444344C3434344A34413463
:100AF0004C3400340034563431342E3430343134F4
:100B0000203420342034303432342E3430343234F3
:100B10002E3431343234003440345634613472343B
:100B2000693461346E3474346534203432342034A2
:100B30002034203420342034203400340034533422
:100B4000613474342D34533475346334683465340B
:100B50002134203420342034203420342034003414
:100B600040344134753466346834653469347A34D9
:100B700065346E3421342034203420340034003481
:100B800054346834653472346D346F34733474346F
:100B90006134743420344C344F345734203420348E
:100BA0000034003454346834653472346D346F3436
:100BB000733474346134743420344F344B342034FF
:100BC0002034203400344034503420340034403455
:100BD000503457344D343A3400344D3453340034A7
:100BE0004D3453342D342D340034003431342E340C
:100BF0004D3465347334733475346E346734213452
:100C00002034203420342034203420340034003484
:100C1000543461347334743465346E3465346934F7
:100C20006E346734613462346534203420342034C7
:100C300000344034543461347334743465342034B3
:100C400031342034203420342034203420342034F3
:100C500020342034003400344D346534733473341C
:100C600075346E3467343A342034203420342034E0
:100C7000203420342034203400344034503457346D
:100C80004D343D3431342034203420342034203469
:100C900020342034203420342034203400344034B4
:100CA000503457344D343D343134323438342034B8
:100CB0002034203420342034203420342034203494
:100CC00000344034503457344D343D3432343534AC
:100CD000353420342034203420342034203420345F
:100CE00020342034003440344E346F3472346D3448
:100CF00061346C347A3475347334743461346E34E2
:100D000064342034203420340034403431343034DE
:100D10002034533465346B34203477346134723486
:100D2000743465346E34203420342034003440343C
:100D3000543461347334743465342034343420349E
:100D40002034203420342034203420342034203403
:100D5000003400345334743461347234743477346E
:100D600065347234743420344E3445345534203470
:100D700020342034003440342034203420342034D3
:100D800020342034203420342034203420342034C3
:100D90002034203420342034003440344C346F3438
:100DA0006334613474346F3472343A342034003430
:100DB00040344E344E343A342034003440344E34CF
:100DC000613476342D344D346F34643465342034DA
:100DD00032344434003440344E34613476342D346B
:100DE0004D346F3464346534203433344434003447
:100DF00040344E34613476342D344D346F346434A1
:100E000065342034533475346334683465340034C5
:100E100000346B34653469346E34653420344634C0
:100E200075346E346B34743469346F346E3400341A
:100E300083018312031789148316031368308F000C
:100E400007308100C33085002F3086008130870055
:100E5000003088000030890080309F0000308E0014
:100E600001308C0000308D000F3095008316031781
:100E700003308800003089008312031360308B0038
:100E8000C33085002F308600813087000030880015
:100E900000308900473090000630920020308400F6
:100EA0008001693004020319572F840A502F8316DA
:100EB0000313A230A100A000831203130800FF3F18
:100EC000FF3FFF3FFF3FFF3FFF3FFF3FFF3FFF3F32
:100ED000FF3FFF3FFF3FFF3FFF3FFF3FFF3FFF3F22
:100EE000FF3FFF3FFF3FFF3FFF3FFF3FFF3FFF3F12
:100EF000FF3FFF3FFF3FFF3FFF3FFF3FFF3FFF3F02
:020000040000FA
:020000040000FA
:04400E00D320FF3F7D
:020000040000FA
:08400000FF3FFF3FFF3FFF3FC0
:020000040000FA
:02401200FF3F6E
:00000001FF
